S1138000CC9BEDCC9BEDCC9BEDCC9BEDCC9BEDCCFC
S11380109BEDCC9BEDCC9BEDCC9BEDCC9BEDCC9B1D
S1138020EDCC9BEDCC9BEDCC9BEDCC9BEDCC9B2484
S1128030CC9B0BCC9BEDCC9BEDCC9BEDCC9BEF79
S11380409B4503FF94CDAC9A9A6E0359C7FFFFA6D4
S113805064CD9B86CD9D5445883DCD9DB5CD9FF97E
S1138060A689CD9CBDCD881BCD9B91CD9D544580CB
S11380707DCD9DB5CD9B91CD8090CC815820202085
S1138080414139303820352E304C002035304C00F9
S113809045808BB685F12617B686AF01F12610B65A
S11380A087AF01F12609B688AF01F12602201BCD66
S11380B0ADB4A6C0CD9CBD4580CBCD9DB51902CD38
S11380C09EFBCD9E11CD9F231802812028757064DC
S11380D06174696E67206D656D2900CD9DF583CC53
S11380E080DFCD9CAB030BFD3F26CD9D5445810520
S11380F0CD9DB545812A35B545813235B735B14E6B
S11381009AB0CC9F3753656C656374204D6F64657A
S11381103A00B69A2603CC8199A1012603CC815852
S1138120A1022603CC8246CC81F0819981588246F3
S113813081F043617061636974616E636500496DC8
S1138140706564616E63650056464F00496E6475E0
S11381506374616E63650000A601B79ACD9CABA6FB
S113816001B758C7012AC7012BC7012C3FFAA60043
S1138170C7012DB69B27036E5426CD8287000B03BF
S1138180CC9738040A03CC94C6020A03CC868C3DEF
S1138190FA2703CCAF7ACC80E2A600B79ACD9CAB89
S11381A0CD9D544581DFCD9DB5CD9B916E01584F3A
S11381B0C7012AC7012BC7012C3FFAA603C7012D0B
S11381C0CD8287000B03CC9738040A03CC94C602F3
S11381D00A03CC868C3DFA2703CCAF7ACC80E243E9
S11381E0617061636974616E63652028704629005B
S11381F0A603B79ACD9CABCD9D54458236CD9DB593
S1138200CD9B916E01584FC7012AC7012BC7012C82
S11382103FFAA604C7012DCD8287000B03CC973803
S1138220040A03CC94C6020A03CC868C3DFA2703C5
S1138230CCAF7ACC80E2496E64756374616E636519
S1138240202875482900A602B79ACD9CABCD9D5431
S11382506E01584FC7012AC7012BC7012C3FFAA64C
S113826001C7012DCD8287000B03CC9738040A0384
S1138270CC94C6020A03CC868C3DFA2703CCAF7A91
S1138280CC80E256464F00CD9D5AB6582710C60101
S11382902A270BA680CD9CBD4583B0CD9DB5CD844A
S11382A058CD84C5B6582703CD9BF0A60ECD9CBDF2
S11382B0A687CD9CBDB658270D4FC70105CDA47226
S11382C0C60103C70102A606B755B756B757020B36
S11382D003CC83AB020A03CC83AB040A03CC83AB89
S11382E0000B03CC83ABCDA06F2705B7FACC83ABCF
S11382F04E0960B660A430B762B8632613B6582737
S1138300CDC6010426C8CD9BF0A601C7010520BE39
S1138310CD9CAB4FC701051763B66349B862B76319
S11383200B6342B655B7563A5727054E6263209EF3
S113833006601755A49FA1012702AFFF35A4D68379
S1138340B5CD9CBD4E6263CC82C655A4CD8432CDDE
S113835084C5CD84583D582706CD9BF0CDA4724EDC
S11383606263CC82C6B655B7573A5627064E626347
S1138370CC82CE06601A55A4AF019FA107972602AE
S1138380AFFF35A4D683B5CD9CBD4E6263CC82C607
S113839055A4CD83BCCD84C5CD84583D582706CD86
S11383A09BF0CDA4724E6263CC82C64FC701058197
S11383B0535752200084858788898B8C35A2C60147
S11383C0602608B670A10327682014A1022608B607
S11383D070A101275C2008B670A10627542000E68E
S11383E070AB01B75FAB062908B65FA40FE7702036
S11383F0406F70AFFF5D26C6C601602700E670A11E
S11384000226BB450000A603201AE670A10526AE8D
S1138410450000A606200DE670A10026A145000037
S1138420A6012000E7709FB1A3270697AF014F2054
S1138430F38135A2E670A0012504E7702019A6098E
S1138440E770AFFF5D26EDE6704D26E855A26F702C
S11384505D2704AFFF20F781CD9CEBA684CD9CBDA6
S1138460CD9CEBB670AA20A1202702AA10CD9CCFE8
S1138470CD9CEBB671AA30CD9CCFCD9CEBA62CCD78
S11384809CCFCD9CEBB672AA30CD9CCFCD9CEBB6E5
S113849073AA30CD9CCFCD9CEBB674AA30CD9CCFC3
S11384A0CD9CEBA62ECD9CCFCD9CEBB675AA30CD42
S11384B09CCFCD9CEBB676AA30CD9CCF55A4D68369
S11384C0B5CD9CBD813F5F3F6B3F6C3F6D3F6E3FC1
S11384D06FC601602708A1022704A601B76F6EAD1D
S11384E0BC6E01BBC601602711A10127086E98BCB0
S11384F06E05BB20056EEFBC3FBB3FBA3FB94E765D
S1138500A1CC86156EC7BC6E10BBC601602712A134
S11385100127086EEDBC6E37BB20066E52BC6E0997
S1138520BB3FBA3FB94E75A1CC86156EC6BC6EA7CB
S1138530BBC601602712A10127086E3EBC6E2FBB8B
S113854020066E35BC6E5DBB3FBA3FB94E74A1CCFC
S113855086156EB9BC6E8DBB6E06BAC6016027184F
S1138560A101270B6E68BC6ED8BB6E15BA20096ECC
S113857011BC6EA4BB6E03BA3FB94E73A1CC861571
S11385806E37BC6E89BB6E41BAC601602718A10163
S1138590270B6E0EBC6E74BB6EDABA20096EADBCCE
S11385A06E68BB6E24BA3FB94E72A120686E29BCB6
S11385B06E5CBB6E8FBA6E02B9C60160271EA10144
S11385C0270E6E89BC6E88BB6E88BA6E08B9200C03
S11385D06EC1BC6E16BB6E6CBA6E01B94E71A12031
S11385E0346E9ABC6E99BB6E99BA6E19B9C60160A5
S11385F0271EA101270E6E55BC6E55BB6E55BA6E73
S113860055B9200C6E8EBC6EE3BB6E38BA6E0EB9D3
S11386104E70A120006E04609836A12403CD865BC1
S11386209839BC39BB39BA39B93B60EC3C5FB65FA9
S1138630A1012603CC8504A1022603CC852BA1032A
S11386402603CC8552A1042603CC8580A1052603EC
S1138650CC85ADA1062603CC85E181B66BBBBCB746
S11386606B240A3C6C26063C6D26023C6EB66CBB41
S1138670BBB76C24063C6D26023C6EB66DBBBAB724
S11386806D24023C6EB66EBBB9B76E81030AFDCD94
S11386909CAB3F26CD9D544586CECD9DB5458720C8
S11386A035B545873E35B735B14EAFB0CD9F37B6FA
S11386B0FF27151902A6C0CD9CBD458701CD9DB5E8
S11386C0CD871118020709FD4FB7FFCC8112436F04
S11386D06E6669672053656C656374696F6E0053D9
S11386E0656C65637420737465702073697A653A88
S11386F0002D20437573746F6D2042616E64202DCC
S1138700002020202028736176696E6729202020AC
S1138710001902CD9EFB180281A60EB7AFCC9109B9
S113872087198DB88DE78E0687FA8D638B0E8B972C
S11387308C208E2D8AA7893388C6884686AF4361EC
S11387406C696272617465004445425547204D6FFF
S1138750646500536F667477617265204C6F616461
S1138760004465627567204D6F6E69746F720042D4
S113877061747465727920566F6C74616765004426
S1138780656661756C745F53657474696E677300B4
S11387904444532053656C656374696F6E0044618F
S11387A07461204F7074696F6E73004C69676874EC
S11387B02053657474696E67730056696577205336
S11387C0657474696E677300546F6E6520536574C5
S11387D074696E677300456E642046726571005358
S11387E0746172742046726571005374657020530D
S11387F0697A6500457869740000A604B7AFCD9D19
S11388005445883DCD9DB5CD9FF9A689CD9CBDCD60
S1138810881B0609F20709FDCC868CB6EAAB30CD7D
S11388209CCFB6EBAB30CD9CCFA62ECD9CCFB6EC77
S1138830AB30CD9CCFB6EDAB30CD9CCF81426174D3
S1138840746572793A00A60DB7AFCD9D544586DFA5
S1138850CD9DB545889935B54588A335B735B14E15
S113886098B0B6B0A1022B04A1072B036E02B03A54
S1138870B03AB0CD9F37CC868C450002201245001B
S113888003200D450004200845000520034500068B
S11388903597A601B7FFCC868C8879887E88838833
S11388A088888D313030206B487A003130206B4815
S11388B07A0031206B487A0031303020487A003118
S11388C03020487A0000A60CB7AF3F58A601C70174
S11388D0224FC7012BCD9D54A6C0CD9CBD458923F5
S11388E0CD9DB54E89704E8A714E8B724E8C734EEF
S11388F08D744E8E754E8F7645000235A4CD89BD9C
S11389004E70894E718A4E728B4E738C4E748D4E9E
S1138910758E4E768FA601B7FFC7012B4FC7012274
S1138920CC868C536574206E6577205374617274A1
S11389303A2000A60BB7AF3F58A601C701224FC784
S1138940012BCD9D54A6C0CD9CBD4589AFCD9DB511
S11389504E90704E91714E92724E93734E94744E2B
S113896095754E967645000235A4CD89BD4E70901E
S11389704E71914E72924E73934E74944E75954E01
S11389807696B670A10326194FB771B791B772B72F
S113899092B773B793B774B794B775B795B776B7FB
S11389A096A601B7FFC7012B4FC70122CC868C5373
S11389B06574206E657720456E643A20000709FDD2
S11389C0CD9D5ACD8458A60ECD9CBDA687CD9CBD09
S11389D04FC70154C70155A606B755B756B7570632
S11389E00905A601C701554E0960B660A430B762F7
S11389F0B863261B0709E8C60154260AC601552791
S1138A00DE4FC70105814FC70154C7015520D0CDA2
S1138A109CAB4FC701051763B66349B862B7630BD4
S1138A20633DB655B7563A5727054E626320B006E4
S1138A30601CA601C7015455A49FA1012702AFFFE2
S1138A4035A4D68AA0CD9CBD4E6263CC89D755A4EB
S1138A50CD8432CD84C5CD84584E6263CC89D7B6DB
S1138A6055B7573A5627064E6263CC89DF06601F16
S1138A70A601C7015455A4AF019FA107972602AFD1
S1138A80FF35A4D683B5CD9CBD4E6263CC89D75542
S1138A90A4CD83BCCD84C5CD84584E6263CC89D724
S1138AA084858788898B8CA60AB7AFCD9D54459061
S1138AB050CD9DB5458ADC35B5458AE035B735B12D
S1138AC04E9BB0CD9F37CC868CA601B79BB7FFCC0D
S1138AD0868C4FB79BA601B7FFCC868C8AC98AD2F5
S1138AE0202020546F6E65204F4E2020202000202F
S1138AF02020546F6E65204F4646202020000054ED
S1138B006F6E652053657474696E67733A00A60EC0
S1138B10B7AFCD9D54459068CD9DB5458B6035B5B7
S1138B20458B6435B735B1C60160B7B0CD9F37CC3E
S1138B30868C4F2006A6012002A602C70160CD9DA7
S1138B4054458B89CD9DB5A6C0CD9CBD458701CD2F
S1138B509DB51902CD9E11CD9F2318029ACC868C07
S1138B608B328B353330204D487A202841443938B4
S1138B703530292020003630204D487A20284144C1
S1138B803938353129202000004444532073656C62
S1138B9065637465642100A607B7AFCD9D54458C09
S1138BA012CD9DB5458BD135B5458BD935B735B18A
S1138BB04E9CB0CD9F37CC868CA600200BA60220FD
S1138BC007A60320039DA601B79CA601B7FFCC8688
S1138BD08C8BB98BBD8BC18BC54E6F204461746186
S1138BE020536176650053656E6420647572696E06
S1138BF067205363616E0053656E642066726F6D07
S1138C00204D656D004461746120746F204D656D65
S1138C10000044617461204F7074696F6E733A0090
S1138C20A608B7AFCD9D54458C4DCD9DB5B69EC716
S1138C300100B69DC70101CD8C5EB79FC60100B788
S1138C409EC60101B79DA601B7FFCC868C4C697402
S1138C5065204F66662F4F6E2054696D6500CD9D6B
S1138C6083A6C0CD9CBD458C9ECD9DB5CD8D03A660
S1138C7004CD9C3F250C2605CD8CD820F2CD8CABA1
S1138C8020EDC60101A40FB7BA3FB96E0ABE3FBDBD
S1138C90CDA142C60100A40FBBBC0709FD814D69EB
S1138CA06E75746573203D20303000C601004AC7DC
S1138CB00100A12F9302201CA639C70100C601019F
S1138CC04AC70101A12F2702200AA639C70100A61D
S1138CD031C70101CD8D0381C601004CC70100A13C
S1138CE03A9002201AA630C70100C601014CC70100
S1138CF001A13227022008A630C70100C70101CD17
S1138D008D0381A6CACD9CBDC60101A130260CC627
S1138D100100A13026022023C60101CD9CCFA6CBA1
S1138D20CD9CBDC60100CD9CCFA6CCCD9CBDA620BC
S1138D30CD9CCFCD9CA5A6FFB7A081A64FCD9CCF3F
S1138D40A6CBCD9CBDA666CD9CCFA6CCCD9CBDA606
S1138D5066CD9CCFCD9CA84FB7A0A630C70101C754
S1138D60010081A60EB7AFCD9D54458D97CD9DB51D
S1138D70CD8E0825094FC701043FFFCC868CCD9DBD
S1138D8054458DA8CD9DB51902CD9E02CDADB4CD6F
S1138D909EFE1802CC868C526573746F72652064D3
S1138DA0656661756C743F002028706C656173653D
S1138DB02077616974292000A60ECD9D54458DDB72
S1138DC0CD9DB5CD8E0825094FC701043FFFCC8644
S1138DD08CA601C701043FFFCC868C44656275678D
S1138DE0204D6F64653F009B45045094CDF2006EA6
S1138DF003196E40136E0C146E031F6E400D6EB893
S1138E003E1D09CCEF2A8381458E1D35B5458E2143
S1138E1035B735B13FB0CC9F34998198818E1B8E84
S1138E201920204E6F0020205965730000A609B751
S1138E30AFCD9D5445902CCD9DB5CD9D83A6C0CD81
S1138E409CBD45903BCD9DB5A6C7450089CD8FE817
S1138E50A605CD9C3F2403CC8FE1CD9D83A6C0CD38
S1138E609CBD459043CD9DB5A6C5450090CD8FE8EA
S1138E70A605CD9C3F2403CC8FE1CD9D83A6C0CD18
S1138E809CBD459049CD9DB5A6C6CD9CBDB698A1C7
S1138E900226054588A32025A10326054588AB2085
S1138EA01CA10426054588B22013A1052605458882
S1138EB0B8200AA1062703CC8FE74588BFCD9DB50E
S1138EC0A605CD9C3F2403CC8FE1CD9D83A6C0CDC8
S1138ED09CBD459050CD9DB5A6C6CD9CBD3D9B2760
S1138EE005459057200345905FCD9DB5A605CD9CC3
S1138EF03F2403CC8FE1CD9D83A6C0CD9CBD45907E
S1138F0068CD9DB5A6C5CD9CBDC60160270EA10147
S1138F10270545907920084590912003459085CDFB
S1138F209DB5A605CD9C3F2403CC8FE1CD9D83A6A2
S1138F30C0CD9CBD4590C2CD9DB5A6CACD9CBDB645
S1138F409CA10026054590D3200CA101260545903F
S1138F50E020034590DACD9DB5A605CD9C3F2403C2
S1138F60CC8FE1CD9D83A6C0CD9CBD4590F8CD9D11
S1138F70B5A6CBCD9CBDB6A027054590AE20034534
S1138F8090B8CD9DB5A605CD9C3F2555CD9D83A616
S1138F90C0CD9CBD4590E7CD9DB5A6CECD9CBDB6BC
S1138FA09DCD9CCFA6CFCD9CBDB69ECD9CCFA60516
S1138FB0CD9C3F252CCD9D83A6C0CD9CBD45909DC9
S1138FC0CD9DB5A6C7CD9CBD3D9B27054590AE2044
S1138FD0034590B8CD9DB5A605CD9C3F2503CC8E09
S1138FE03A0709FDCC868C83CD9CBDF6AA30CD9C76
S1138FF0CFAF01F6AA30CD9CCFA62CCD9CCFAF012C
S1139000F6AA30CD9CCFAF01F6AA30CD9CCFAF01EC
S1139010F6AA30CD9CCFA62ECD9CCFAF01F6AA30B8
S1139020CD9CCFAF01F6AA30CD9CCF81557365722C
S11390302053657474696E67733A00537461727473
S11390403A2000456E643A2000537465703A20005B
S1139050546F6E653A2000656E61626C65640064ED
S1139060697361626C6564004444533A2020202093
S11390702020202020202020003130204D487A203C
S113908020202020003330204D487A20202020202A
S1139090003630204D487A2020202020004465628C
S11390A075673A20202020202020202020006F6E89
S11390B020202020202020006F66662020202020F1
S11390C02000446174614D6F64653A2020202020A3
S11390D02020004E6F4461746100546F205043009F
S11390E0546F204D656D004C6974654F666620545D
S11390F0696D65723A2020004261636B6C69676830
S1139100743A202020202020009BCD93D1A600B7C4
S1139110FFC7012DCD9D54459462CD9DB5CD8E08DC
S11391202503CC868CCD9D54459471CD9DB5CD8EB3
S1139130082503CC868CCD9BA3A602CD9C8CC701AD
S113914056A600CD9C8CC70158A601CD9C8CC701A6
S113915059A604CD9C8CC70157CD93E0CD9D5445B1
S11391609451CD9DB5A6C0CD9CBDA602CD9C8CCD01
S113917093C4A6C4CD9CBDA600CD9C8CCD93C4A69F
S1139180C8CD9CBDA601CD9C8CCD93C4A6CCCD9C52
S1139190BDA604CD9C8CCD93C40609C90709FDCD99
S11391A09D5445947CCD9DB5CD8E082503CC868CED
S11391B0CDA051A602CD9C8CCDA3FBB7BC3FBB3F39
S11391C0BA3FB9C60156CDA3FBB7C03FBF3FBE3FB0
S11391D0BDCDA378B6BCCDA3FBB7BE3FBD6E64BA0C
S11391E03FB9CDA14245010ACD9384CDA41AA6046A
S11391F0CD9C8CCDA3FBB7BC3FBB3FBA3FB9C601E6
S113920057CDA3FBB7C03FBF3FBE3FBDCDA378B68C
S1139210BCCDA3FBB7BE3FBD45010ACD93A4CDA2EF
S113922040B6BCC7015ACDA3FBA672CDA05DB6BEA5
S1139230C7015BCDA3EEA600CD9C8CCDA3FBB7BC30
S11392403FBB3FBA3FB9C60158CDA3FBB7C03FBF30
S11392503FBE3FBDCDA378B6BCCDA3FBB7BE3FBDDB
S113926045010ACD93A4CDA240B6BCC7015CCDA3F1
S1139270FBA672CDA05DB6BEC7015DCDA3EECD9DAC
S113928054459497CD9DB5CD8E082503CC868CCDC1
S11392909D5445948ACD9DB5CDA4AEA601CD9C3FE9
S11392A025142609C6015C4CC7015C20EBC6015C91
S11392B04AC7015C20E2C6015CCDA3FBA672CDA027
S11392C05DB6BEC7015DCDA3EE0709FDCD9D544536
S11392D094A8CD9DB5CD8E082503CC868CA602CD51
S11392E09C8CCDA3FBB7BC3FBB3FBA3FB9C601566C
S11392F0CDA3FBB7C03FBF3FBE3FBDCDA378B6BC37
S1139300CDA3FB4EBCBE4EBBBD6E32BA3FB9CDA1A0
S11393104245010ACD9384CDA41AA601CD9C8CCDDF
S1139320A3FBB7BC3FBB3FBA3FB9C60159CDA3FBB2
S1139330B7C03FBF3FBE3FBDCDA378B6BCCDA3FBF6
S1139340B7BE3FBD45010ACD93A4CDA240B6BCC76C
S1139350015ECDA3FBA672CDA05DB6BEC7015FCDF5
S1139360A3EECD9D544594B8CD9DB5A6C0CD9CBD6E
S1139370458701CD9DB51902CD9E11CD9F231802BD
S11393809ACC868CB6B9F7B6BAE701B6BBE702B693
S1139390BCE70381B6BDF7B6BEE701B6BFE702B6C8
S11393A0C0E70381F6B7B9E601B7BAE602B7BBE690
S11393B003B7BC81F6B7BDE601B7BEE602B7BFE6A8
S11393C003B7C081CDA03F8B86CD9CCF9FCD9CCFD2
S11393D081C601602605459429201D459441201825
S11393E0C60160270EA1012705459439200A45943A
S11393F03120054594492000F6B76FE601B76EE6C3
S113940002B76DE603B76CE604B76BE605B770E622
S113941006B771E607B7723F733F743F753F76CD69
S11394209BF0CD9BF0CD9BF081010000000000007B
S113943000010E38E38E010000005555555501001A
S1139440000000000000000000001999999A010032
S1139450005646202056522020565A20205641209D
S1139460200043616C696272617465206E6F773F9E
S1139470004F70656E206C6F61643F0053686F72BB
S1139480746564206C6F61643F004D616B652053AB
S113949057523D352E34003237302D6F686D206CB5
S11394A06F6164206F6E3F0035302D6F686D206CE6
S11394B06F6164206F6E3F0043616C20636F6D7059
S11394C06C6574652100050AFDCD9CAB3F58CD9BAE
S11394D0A3CD9D544595ACCD9DB5A6C0CD9CBD45B1
S11394E095BDCD9DB56E00E36E01E46E00E56E00A2
S11394F0E66E00E76E00E86E00E96E09E16E09E2CF
S11395004E77704E78714E79724E7A734E7B744EEC
S11395107C754E7D766E703A1902CD95CDCD84C59D
S1139520CD9BF0CDA4AECD9706CD96185597CD839F
S1139530BCCD84C5CD9BF0CDA4AECD9706CD9618F9
S1139540050A49B670B07E26E3B671B07F26DDB653
S113955072B08026D7A602B1982731B673B081269F
S1139560CBA603B1982725B674B08226BFA604B152
S1139570982719B675B08326B3A605B198270DB6FA
S113958076B08426A7A606B198270183CD969318B2
S113959002050AFD4EE3704EE4714EE5724EE67329
S11395A04EE7744EE8754EE976CC81587E7E7E2077
S11395B05343414E4E494E47207E7E7E0020202854
S11395C0706C6561736520776169742900B69CA12C
S11395D0012705A10227028181CD967E450077A649
S11395E006AD18CDA05145007EA606AD0ECDA05106
S11395F0450097A602AD04CDA0518187B69CA10178
S11396002706A1022704868186818687F6CD96A83F
S1139610AF019E6B01F68681B69CA1012705A102CC
S11396202702818155D335BBCDA0A2B6EDCD96A836
S1139630A62ECDA05DB6EECD96A8B6EFCD96A8A683
S11396402CCDA05DCDA762CDA7A255DB35BBCDA0A7
S1139650A24500ECA604CD95FBA62CCDA05DCDA91A
S11396607555F435BBCDA0A24500ECA603CD95FB02
S1139670A62ECDA05DB6EFCD96A8CDA05181B69C07
S1139680A1012705A10227028181A653CDA05DCDAA
S1139690A05181B69CA1012705A10227028181A6C0
S11396A045CDA05DCDA05181A40FAB30A1392302DB
S11396B0AB0787B69CA1012706A1022704868186F1
S11396C08186CCA05DA686CD9CBDB6E3AA30CD9C98
S11396D0CFB6E4AA30CD9CCFA62CCD9CCFB6E5AABC
S11396E030CD9CCFB6E6AA30CD9CCFB6E7AA30CD1C
S11396F09CCFA62ECD9CCFB6E8AA30CD9CCFB6E9A0
S1139700AA30CD9CCF81B6DFB1E12607B6E0B1E245
S11397102504812501814EDFE14EE0E24E70E34EE7
S113972071E44E72E54E73E64E74E74E75E84E767C
S1139730E9C60102C7010381010BFDCD9CAB3F26A5
S1139740CD9BA3CD9D54459988CD9DB5459A3F3574
S1139750B5459A5D35B735B14E99B0CC9F3745972D
S11397606BCD98F2A600B799CC995802000000007E
S1139770000003000000000000459786CD98F2A683
S113978001B799CC995801000000000000020000C4
S1139790000000004597A1CD98F2A602B799CC9994
S11397A05800010000000000010000000000004516
S11397B097BCCD98F2A604B799CC9958000108003B
S11397C0000000000200000000004597D7CD98F289
S11397D0A605B799CC9958000305000000000004C1
S11397E000000000004597F2CD98F2A606B799CC88
S11397F09958000700000000000007030000000063
S113980045980DCD98F2A607B799CC995801000157
S11398100000000001000105000000459828CD98D3
S1139820F2A608B799CC9958010400000000000181
S1139830040305000000459843CD98F2A609B799A2
S1139840CC99580108000608000001080106080028
S11398500045985ECD98F2A60AB799CC99580201B2
S1139860000000000002010405000000459879CDC5
S113987098F2A60BB799CC99580204080900000085
S113988002040909000000459894CD98F2A60CB78B
S113989099CC995802080000000000020907000052
S11398A00000C601602607A60CB799CC97384598E6
S11398B0BBCD98F2A60DB799CC99580500000000CD
S11398C0000005040000000000C60160A101270794
S11398D0A600B799CC97384598E4CD98F2A60EB770
S11398E099CC995803000000000000060000000015
S11398F00000F6B777E601B778E602B779E603B772
S11399007AE604B77BE605B77CE606B77DE607B7DB
S11399107EE608B77FE609B780E60AB781E60BB7AB
S113992082E60CB783E60DB78481A603B7994E8906
S1139930774E8A784E8B794E8C7A4E8D7B4E8E7C08
S11399404E8F7D4E907E4E917F4E92804E93814EEF
S113995094824E95834E96840709FD4E77E34E77A5
S1139960704E78E44E78714E79E54E79724E7AE60F
S11399704E7A734E7BE74E7B744E7CE84E7C754E7C
S11399807DE94E7D76CC811242616E642053656C14
S1139990656374696F6E0042616E643A20312D31E3
S11399A030204D487A0042616E643A2031302D32C5
S11399B030204D487A0042616E643A2032302D33B3
S11399C030204D487A0042616E643A203136306D61
S11399D00042616E643A202038306D0042616E644A
S11399E03A202034306D0042616E643A20203330D6
S11399F06D0042616E643A202032306D0042616E27
S1139A00643A202031376D0042616E643A2020317F
S1139A10356D0042616E643A202031326D0042613E
S1139A206E643A202031306D0042616E643A202029
S1139A30366D00437573746F6D2042616E640097D8
S1139A405E97799794992A97AF97CA97E598009863
S1139A501B98369851986C988798A298C932302DE3
S1139A603330204D487A0031302D3230204D487A41
S1139A7000312D3130204D487A00437573746F6D79
S1139A802042616E64003136306D2042616E6400A4
S1139A902038306D2042616E64002034306D2042E5
S1139AA0616E64002033306D2042616E64002032A8
S1139AB0306D2042616E64002031376D2042616E4A
S1139AC064002031356D2042616E64002031326DB6
S1139AD02042616E64002031306D2042616E64006A
S1139AE02020366D2042616E640033302D363020E4
S1139AF04D487A00006E36206E002A6E882B6E0068
S1139B00276E41286E54296E0620818B89871F2673
S1139B1055279FCB01029724058B9E6C018A35271C
S1139B2086888A808B89871F29552AAF7FAF09359C
S1139B302A3D5927073A592603CD9B53555A2704E2
S1139B40AFFF355A55F2AFFF35F22603CD9B74862D
S1139B50888A80C60105270DCDA472C6012DA100F7
S1139B602603CDAE40A6FFB7590D09031D09811C7C
S1139B7009819D8145EA6035F2C601204AC701206A
S1139B802603CD9CA88187A6164BFE9E6B01F88602
S1139B9081A60AB7A9A650B7A8CD9BD83BA8FA3B83
S1139BA0A9F381A66487AD30864BFA81A64087ADC0
S1139BB027864BFA816E32593D5926FC81A62087AF
S1139BC0AD16864BFA81A61087AD0D864BFA81A699
S1139BD00A87AD04864BFA81A60A87AD04864BFA40
S1139BE081A6AE4A9D26FC81B6034BFE819D8081F1
S1139BF045006B6E056A7E696E0868366924081034
S1139C00091209130920061109120913093B68EB0B
S1139C103B6AE31409150981C601602712A10227D2
S1139C200E1209130914091509CD9C30CD9C3081FD
S1139C303F6B3F6C3F6D3F6E6E016FCD9BF081B704
S1139C4055B756B7579D0709410A09083D652707C7
S1139C503F6520116EFF650909056EFF6620E63D2C
S1139C606627E23F664E6263B609A430B762B86302
S1139C70A410270BB655B7573B56CAA6019881B610
S1139C8055B7563B57BFA60098819981B7380F380E
S1139C90FDB63981A600CD9C8CC70102A6FFC00188
S1139CA002C7010281140281150281B69FC70120F7
S1139CB0B6A02705CD9CA52003CD9CA881B75E1333
S1139CC000CD9CEB17006EFF07150013002010B7A2
S1139CD05E1200CD9CEB17006EFF0715001200B654
S1139CE05EB7031600CD9BE81700814F6E0F071374
S1139CF0001400CD9BE86EFF5C1600CD9BE84E037C
S1139D005D17003B5C0220030E5DEE81150013001D
S1139D10CD9BA36E30031600CD9BE81700CD9BCFDF
S1139D206E30031600CD9BE81700CD9BCF6E300339
S1139D301600CD9BE81700CD9BCFA63CCD9CBDA6BD
S1139D4008CD9CBDA601CD9CBDA606CD9CBDA60C90
S1139D50CD9CBD81A601CD9CBD81A680CD9CBDCDF1
S1139D609BD8459D6ECD9DB5A680CD9CBD81202000
S1139D7020202020202020202020202020202020DF
S1139D80202000A6C0CD9CBDCD9BD8459D6ECD9D09
S1139D90B5A6C0CD9CBD81A608CD9CBD81A60CCD29
S1139DA09CBD81A60FCD9CBDCD9BD881A60CC69C25
S1139DB0BDCD9BD881F62707CD9CCFAF0120F6817E
S1139DC087CD9E20A61843C4FE1DC7FE1DAA04C746
S1139DD0FE1D86F7A601CAFE1DC7FE1DCD9BA3A6C8
S1139DE00143C4FE1DC7FE1DCD9BE1A60443C4FE72
S1139DF01DC7FE1D81450800C6FE1DAA18C7FE1D0D
S1139E002028450800C6FE1DA4F7AA10C7FE1D2081
S1139E1019450880C6FE1DA4FEAA10C7FE1D200A0F
S1139E20C6FE1DA4EFAA08C7FE1DAA04C7FE1DF79F
S1139E30A601CAFE1DC7FE1DCD9BA3A60143C4FEF9
S1139E401DC7FE1DCD9BE1A60443C4FE1DC7FE1D18
S1139E5081CD9E6EA61045FE1CCD9DC0F6A6804504
S1139E60FE10CD9DC0A6AC45FE11CD9DC081A6209F
S1139E7043C4FE1DC7FE1D81C6FE1DAA20C7FE1DCC
S1139E80814E1061336145FE1CF6B461CD9DC081E5
S1139E9045FE1CF6AA10CD9DC0F681A40FB76145FE
S1139EA0FE1CF6BA61CD9DC0F681A40F43B761458F
S1139EB0FE1CF6B461CD9DC0F681C60800A1FF2644
S1139EC007CD9EFBCD9F238145080035AC45008519
S1139ED035AA6E1CAECD9EE945088035AC450156C9
S1139EE035AA6E0BAECD9EE98155ACF6AF0135AC0B
S1139EF055AAF7AF0135AA3BAEEF81CD9E024508C6
S1139F000035AA45008535AC6E1CAECD9F0F81553A
S1139F10ACF6AF0135AC55AACD9DC0AF0135AA3B17
S1139F20AEED8145088035AA45015635AC6E0BAEC1
S1139F30CD9F0F81CC9FA14500B07D2719B6B055A8
S1139F40B17D2704AF0120F94A2707AF017D270D12
S1139F5020EFAF01276255B1CD9CAB205BCC9FEDC8
S1139F60A60ACD9C3F25622638CD9CAB55B1CD9F2A
S1139F70EE26277D2704AF0120F93CB0AF017D26F2
S1139F80F2AFFF7D2667AFFF7D2707CD9FEE26F654
S1139F902002AF013AB02B55201EAFFF7D264E2084
S1139FA0E5CD9CAB55B17D2704AF0120F93CB0AFA2
S1139FB0017D26043FB055B735B1CD9D83A6C0CDF4
S1139FC09CBD55B1CD9DB52097CD9CAB55B507092A
S1139FD0FD8B89B6B09849B76186BB61B76186A924
S1139FE000878AB66197F687E601978AFC839FB15A
S1139FF0B82701818B86B1B781A603CD9C8CB7BAF3
S113A0003FB96EC3BE3FBDCDA1423FBD3FBE6E272B
S113A010BF6E10C0CDA1A14EBDB94EBEBA4EBFBBDE
S113A0204EC0BC6E0CBD6E35BECDA240CDA0A2CD3F
S113A030A40581CCF4DBCCF4EECCF53FCCF54DCCCF
S113A040F556CCF561CCF56CCCF577CCF57CCCF53C
S113A05081CCF586CCF58FCCF592CCF599CCF59CDA
S113A060CCF5A5CCF5ADCCF5B9CCF5BDCCF5BECCD5
S113A070F5CDCCF5D7CCF5E1CCF5F6CCF602CCF6A3
S113A0800ACCF60ECCF62ECCF641CCF64ACCF660D1
S113A090CCF66CCCF677CCF67ECCF686CCF689CCB6
S113A0A0F6FA898BB6BC97B6BB878AB6BA2749A19C
S113A0B0012732A102271AA1032702203B6E01EADD
S113A0C06E09EB6E06EC6E06ED6E00EE6E05EF208B
S113A0D0336E01EA6E03EB6E01EC6E00ED6E07EE7B
S113A0E06E00EF201F3FEA6E06EB6E05EC6E05ED89
S113A0F06E03EE6E05EF200C3FEA3FEB3FEC3FEDC5
S113A1003FEE3FEF650000273365000A252EAFF6CA
S113A1103CEEB6EEA10A26EC3FEE3CEDB6EDA10A0C
S113A12026E23FED3CECB6ECA10A26D83FEC3CEB32
S113A130B6EBA10A26CE3FEB3CEA20C89FB7EF8AD4
S113A140888187898BA7FA9E6F06BEBAB6BE429EE7
S113A150EF06B7BCBEB9B6BE429EEB069EE702242C
S113A160015C9EEF019E6F06BEBAB6BD429EEF062D
S113A1709EE705BEB9B6BD429EEB069EE7042401E8
S113A1805C9EEF039EE6029EEB05B7BB9EE6019E36
S113A190E904B7BA9EE603A900B7B9A7068A888678
S113A1A08187898B5F4FA7DD95AF2035DDAFE07FD9
S113A1B05C75DD26FA9EE723A6039EE7219EE7222F
S113A1C095AF0735DD8C9EEE21E6BD9EEE22EEB9FD
S113A1D0429EEB2324015C9EEF2355DDF7AFFF3550
S113A1E0DD8C9E6A222ADF55DD9EE623F7AF0B3510
S113A1F0DD8C9E6F23AE039EEF229E6A212AC795B3
S113A200AF0735DD9E6F23A6079EE721A6039EE7D1
S113A210229EE6239E6F23FB24039E6C23AF089E9D
S113A2206A222AF38CAE039EEF229EEE21E7B955F3
S113A230DDAFFF35DD9E6A212AD7A7238A88868170
S113A2408B8789A7FDA6209EE703B6BD9EE701B6CE
S113A250BE9EE7024EBCBE4EBBBD4EBABC4EB9BBA1
S113A2603FB93FBAB6B94939BE39BD39BC39BB3932
S113A270BA39B9B6BA9EE002B7BAB6B99EE201B726
S113A280B9B6BEA200B7BE01BE16B6BA9EEB02B7FF
S113A290BAB6B99EE901B7B9B6BEA900B7BE2002E5
S113A2A010BE9E6B03BEB6B99EE701B6BA9EE70226
S113A2B04EBBB94EBCBA4EBDBB4EBEBC9EE601B74A
S113A2C0BD9EE602B7BEA70388868A81A7FCB6B9FD
S113A2D09EE701B6BA9EE702B6BB9EE703B6BC9EF4
S113A2E0E7049FB7F18B86B7F0AD0BAD09AD07ADB1
S113A2F005AD03A704819EE603B7B99EE604B7BA89
S113A3009EE605B7BB9EE606B7BC3FBD3FBE3FBF5A
S113A3106E64C0CDA1A14EBDB94EBEBA4EBFBB4EF8
S113A320C0BC4EF0BD4EF1BECDA2404EF0BF4EF1CA
S113A330C03FBD3FBECDA3473FBD6E02BECDA240D0
S113A3404EBBF04EBCF181B6BCBBC0B7BC240A3CCA
S113A350BB26063CBA26023CB9B6BBBBBFB7BB247E
S113A360063CBA26023CB9B6BABBBEB7BA24023C14
S113A370B9B6B9BBBDB7B981B6BCB0C0B7BCB6BB82
S113A380B2BFB7BBB6BAB2BEB7BAB6B9B2BDB7B947
S113A3908187898BC601044D2717B6FBCDA054B61F
S113A3A0FCCDA054B6FDCDA054B6FECDA054CDA096
S113A3B0518A88868187898B8B86CDA0549FCDA0B6
S113A3C0548A88868187898BC601044D27099EE6B5
S113A3D003CDA054CDA0518A88868187898BC6017C
S113A3E0044D27069EE603CDA0548A88868187897A
S113A3F08BCDA054CDA0518A88868187898BCDA02E
S113A400548A88868187898BC601044D27084500B4
S113A410B9AD2BCDA0518A88868187898B4500B937
S113A420AD1CCDA0518A88868187898BC601044DD5
S113A43027084500BDAD07CDA0518A888681898B48
S113A440F6CDA06C8A88898BE601CDA06C8A8889B8
S113A4508BE602CDA06C8A88898BE603CDA0548A52
S113A460888187898BC601044D2703CDA0518A8832
S113A4708681CDA4AECDA762CDA7A2CDA975C60114
S113A4802DA1042605CDAA86201BA1032608CDAB49
S113A490712012C6012DA101260BA6C6CD9CBD4577
S113A4A08283CD9DB555A4D683B5CD9CBD81A6022E
S113A4B0CD9C8CB7FBCDA3DBB7BC3FBB3FBA3FB948
S113A4C0C60156CDA3DBB7C03FBF3FBE3FBDCDA342
S113A4D078B6BCCDA3C54EBCBA4EBBB96E64BE3F04
S113A4E0BDCDA142CDA40545010ACD9384A600CDDE
S113A4F09C8CB7FCCDA3DBB7BC3FBB3FBA3FB9C60E
S113A5000158CDA3DBB7C03FBF3FBE3FBDCDA3784D
S113A510B6B92A083FB93FBA3FBB3FBCB6BCCDA3CE
S113A520DB4EBCBA4EBBB9C6015CCDA3C5B7BE3FBA
S113A530BDCDA142CDA40545010ECD9384CD9C94FF
S113A54045010ACD93A445010ECD93B4CDA3476E26
S113A55064C03FBF3FBE3FBDCDA1A14EBDB94EBEFD
S113A560BA4EBFBB4EC0BCCDA405450117CD9384E4
S113A57045010ACD93A445010ECD93B4CDA378CD66
S113A580A40545011BCD9384B6B9A1FF260F3FB99D
S113A5903FBA3FBB6E02BC45011BCD9384450117F6
S113A5A0CD93A4C6011EB7BEC6011DB7BDCDA24042
S113A5B04500D1CD9384CDA405A604CD9C8CB7FED3
S113A5C0CDA3DBB7BC3FBB3FBA3FB9C60157CDA350
S113A5D0DBB7C03FBF3FBE3FBDCDA378B6BCCDA364
S113A5E0DB4EBCBA4EBBB945011BCD9384C6015AA0
S113A5F0CDA3DBC6015BCDA3C5C6015AB7BE3FBD23
S113A600CDA142450117CD9384C6015BB7BA3FB9CA
S113A610C6011DB7BDC6011EB7BECDA1424EBBBC0F
S113A6204EBABB4EB9BA3FB9450117CD93B4CDA3C9
S113A63047CDA405450106CD9384A601CD9C8CB7D6
S113A640FDCDA3DBB7BC3FBB3FBA3FB9C60159CD73
S113A650A3DBB7C03FBF3FBE3FBDCDA378B6BCCDE3
S113A660A3DB4EBCBA4EBBB945011BCD9384C601D6
S113A6705ECDA3DBC6015FCDA3C5C6015EB7BE3FF9
S113A680BDCDA142450117CD9384C6015FB7BA3F42
S113A690B9C6011DB7BDC6011EB7BECDA1424EBB92
S113A6A0BC4EBABB4EB9BA3FB9450117CD93B4CD30
S113A6B0A347CDA405450112CD93843DD126703D19
S113A6C0D2266C898B55D36503DE8A8824614500C4
S113A6D0D1CD93A4CDA0A24EEDDF4EEEE0B6EFA116
S113A6E0052704240220143CE0A60AB1E0260C3F0E
S113A6F0E03CDFA60AB1DF260220343D5826018162
S113A700C60122270181C6012A260181A6C0CD9C4B
S113A710BDB6DFCDA042CD9CCFA62ECD9CCFB6E05A
S113A720CDA042CD9CCF55A4D683B5CD9CBD81454B
S113A73003DE35D33D582725C6012A2720C601222A
S113A740261BA6C0CD9CBD45A75ECD9DB555A4D600
S113A75083B5CD9CBDA609B7EDB7EEB7EF813E3109
S113A7603000C60115B7BAC60114B7B96E32BE3F80
S113A770BDCDA142C60109B7BEC60108B7BDCDA271
S113A78040CDA4053DB926143DBA2610898B55BB8E
S113A7906502588A8824054FC7011681A601C7019E
S113A7A016814EBCBE4EBBBD4EBEBA4EBDB9CDA188
S113A7B0424EB9C54EBAC64EBBC74EBCC8CDA405A1
S113A7C03FBD3FBE6E09BF6EC4C0CDA3473FBD3F72
S113A7D0BE3FBF6E02C0CDA1A14500D1CD93A4CD93
S113A7E0A1A14EBDC94EBECA4EBFCB4EC0CCCDA456
S113A7F0294ED1B94ED2BA4ED3BB4ED4BC4ED1BDE4
S113A8004ED2BE4ED3BF4ED4C0CDA1A13FB93FBAA4
S113A8106E27BB6E10BCCDA3474500D5CD9384CD28
S113A820A40555D52729B6D526134ECBBC4ECABB95
S113A8304EC9BA3FB94ED7BE4ED6BD20244ECABC6F
S113A8404EC9BB3FBA3FB94ED6BE4ED5BD20124EFF
S113A850CCBC4ECBBB4ECABA4EC9B94ED8BE4ED7ED
S113A860BDCDA2404EB9D94EBADA4EBBDB4EBCDCEC
S113A870CDA405C6011627224FB7D9B7DAB7DBB77F
S113A880DCC6012B270BA6C3CD9CBD45A952CD9D8B
S113A890B555A4D683B5CD9CBD813DB9260A3DBA34
S113A8A02606A608B1BB24123FD93FDA6E08DB3F67
S113A8B0DC3FB93FBA6E08BB3FBCC6012227018109
S113A8C0C6012B260181CDA0A2A6C7CD9CBD45A95A
S113A8D06FCD9DB53D582716A6C3CD9CBD45A96037
S113A8E0CD9DB5A6CACD9CBDC60121CD9CCFA6C524
S113A8F0CD9CBDB6EC4D2604A6202003CDA042CDB0
S113A9009CCFA6C6CD9CBDB6ED4D2609B6EC4D2612
S113A91004A6202005B6EDCDA042CD9CCFA6C7CD80
S113A9209CBDB6EE4D260DB6ED4D2608B6EC2604BC
S113A930A6202005B6EECDA042CD9CCFA6C8CD9CC6
S113A940BDB6EFCDA042CD9CCF55A4D683B5CD9C4A
S113A950BD81202020205A3E363030202020200087
S113A960202020202020202B6A20202020200020AE
S113A97020202020004EDBBD4EDCBE4EDBB94EDC79
S113A980BACDA142CDA405B6C8B0BCB7BCB6C7B257
S113A990BBB7BBB6C6B2BAB7BAB6C5B2B9B7B9CD0A
S113A9A0A405C60116270F450064CDA2CC450000BE
S113A9B035F4CDA405810FB93AC6012C272CA6CCB9
S113A9C0CD9CBDA620CD9CCFA620CD9CCFA620CDCE
S113A9D09CCFA630CD9CCF3FB93FBA3FBB3FBCCD47
S113A9E0A405CDA46245000035F455A4D683B5CDA5
S113A9F09CBD81450064CDA2CC55BB35F4CDA405E6
S113AA00CDA462C60122270181C6012C260181CD75
S113AA10A0A2B6EEB7EFB6EDB7EEB6ECB7EDB6EB77
S113AA20B7ECA6CCCD9CBDB6EC4D2604A6202003E5
S113AA30CDA042CD9CCFA6CDCD9CBDB6ED4D260973
S113AA40B6EC4D2604A6202005B6EDCDA042CD9C43
S113AA50CFA6CECD9CBDB6EE4D260DB6ED4D260847
S113AA60B6EC2604A6202005B6EECDA042CD9CCFA0
S113AA70A6CFCD9CBDB6EFCDA042CD9CCF55A4D6DC
S113AA8083B5CD9CBD81C60116270EA6C6CD9CBD3F
S113AA9045AB57CD9DB5CCAB4E55F465000A241D8E
S113AAA0A6C3CD9CBDA64CCD9CCFA63DCD9CCFA628
S113AAB020CD9CCF45AB64CD9DB5CCAB4E55F43584
S113AAC0BB3FBA3FB93FBD6E01BE6E86BF6EA0C02C
S113AAD0CDA1A14EBDB94EBEBA4EBFBB4EC0BC6ED9
S113AAE002BD6E74BECDA240CDAF2B650000260E14
S113AAF0A6C6CD9CBD45AB64CD9DB5CCAB4E35BD96
S113AB00CDA240CDA0A2A6C3CD9CBDA64CCD9CCFCA
S113AB10A63DCD9CCFA620CD9CCFB6ECCDA042CDFA
S113AB209CCFB6EDCDA042CD9CCFB6EECDA042CD0C
S113AB309CCFA62ECD9CCFB6EFCDA042CD9CCFA668
S113AB4020CD9CCFA675CD9CCFA648CD9CCF55A437
S113AB50D683B5CD9CBD81285A3E3630302920207D
S113AB602020200028583D3029202020202020208B
S113AB7000C60116270EA6C6CD9CBD45AB57CD9D7C
S113AB80B5CCAC6E55F465000A241DA6C3CD9CBD9E
S113AB90A643CD9CCFA63DCD9CCFA620CD9CCF4532
S113ABA0AB64CD9DB5CCAC6E3FB93FBA6E27BB6EDE
S113ABB010BC3FBD6E3FBECDA240450117CD93846E
S113ABC0CDAF2B650000260EA6C6CD9CBD45AC7747
S113ABD0CD9DB5CCAC6E35BD3FB96E01BA6E86BBAA
S113ABE06EA0BCCDA240450117CD93B4CDA1A14523
S113ABF00117CD93943FB93FBA6E27BB6E10BC5575
S113AC00F435BDCDA240450117CD93B4CDA1A14EDD
S113AC10BDB94EBEBA4EBFBB4EC0BCCDA0A2A6C3EA
S113AC20CD9CBDA643CD9CCFA63DCD9CCFA620CD2B
S113AC309CCFB6EACDA042CD9CCFB6EBCDA042CD01
S113AC409CCFB6ECCDA042CD9CCFB6EDCDA042CDED
S113AC509CCFA62ECD9CCFB6EECDA042CD9CCFA648
S113AC6020CD9CCFA670CD9CCFA646CD9CCF55A41D
S113AC70D683B5CD9CBD8128583D30292020202085
S113AC80202020004500213FB93FBA3FBB6E73BC72
S113AC90CDA2CCCDA405CDA462816E0F046E0005B7
S113ACA06E34066EFF076E050C6E470D6E000E6E59
S113ACB0000F6EFF006EFB026EFF036EFB081509AA
S113ACC013091109B609A430B763B7626EFF656E44
S113ACD0FF666E01706E00716E00726E00736E001E
S113ACE0746E00756E007645000335A46E00776EB1
S113ACF001786E00796E007A6E007B6E007C6E00C7
S113AD007D6E017E6E007F6E00806E00816E00821B
S113AD106E00836E0084CDAE1D6E703A4FC7010481
S113AD204FC70105B7FFC70122A60EB7AFA600C7DC
S113AD30012D45000035F4A601C7012AC7012BC720
S113AD40012CA62BC70121CD9E51CD9D0C06090FC8
S113AD50CD9DF5CD9D5445ADA4CD9DB50709FDCD43
S113AD60ADB4CD9D5445AD94CD9DB51902CD9EBADB
S113AD701802B69FC70120B6A027041402200215AA
S113AD800245EA6035F2CD9AF5CDAE39CD9C184F27
S113AD90C7015081496E697469616C697A696E672B
S113ADA02E2E2E00454550524F4D20636C65617226
S113ADB06564210045808BF6B785AF01F6B786AF91
S113ADC001F6B787AF01F6B7886E00896E058A6E03
S113ADD0008B6E008C6E008D6E008E6E008F6E0187
S113ADE0906E02916E00926E00936E00946E0095C8
S113ADF06E00964500033597A601B799A601B79A48
S113AE004FB79BA600B79CA630B79DA631B79EA6A8
S113AE1001B79FA601B7A0A600C70160816E01E338
S113AE206E00E46E00E56E00E66E00E76E00E86E0C
S113AE3000E96E09E16E09E2813F593F5A3F5B81A7
S113AE40010A06A620C701218155F435F6CDAEE6E8
S113AE50B6702709A1032742A102273E9D450001A0
S113AE60CD83BC450001CD83BC450001CD83BCCD61
S113AE7084C5CD9BF0CD9BCFA601C70122CDA47282
S113AE8055F49FB0F78B86B2F62407A62DC701218F
S113AE902042A62BC70121CCAED4450001CD84327B
S113AEA0450001CD8432450001CD8432CD84C5CD29
S113AEB09BF0CD9BCFA601C70122CDA47255F49F70
S113AEC0B0F78B86B2F62407A62BC701212005A66E
S113AED02DC70121CDAF0CCD84C5CD9BF04FC7014B
S113AEE02255F635F481450070F6C70123E601C703
S113AEF00124E602C70125E603C70126E604C701CB
S113AF0027E605C70128E606C7012981450123F67E
S113AF10B770E601B771E602B772E603B773E604E9
S113AF20B774E605B775E606B77681450000B670D6
S113AF302706CDAF6D4A26FAB6712706CDAF604A13
S113AF4026FAB6722705AF644A26FBB6732705AF07
S113AF500A4A26FBB6742705AF014A26FB35F88159
S113AF60879FABE8978B86A903878A8681879FABE7
S113AF7010978B86A927878A8681B6FAA0302B3A48
S113AF8048A11A903545AFBD898B9EEB029EE7021E
S113AF909EE601A9009EE7018A88F6EE01878ACD24
S113AFA098F24E77E34E78E44E79E54E7AE64E7B9E
S113AFB0E74E7CE84E7DE9CC94C6CC815897A197A6
S113AFC086976B008998949879985E984398289806
S113AFD00D97F297D797BC4E89774E8A784E8B7926
S113AFE04E8C7A4E8D7B4E8E7C4E8F7D4E907E4E57
S113AFF0917F4E92804E93814E94824E95834E96CD
S113B00084811310180C6E001118086E2010121091
S113B0108119080711FD6E06120711FD0F11FDB607
S113B02012180881CDB0B487A4018626F781F6876B
S113B030AF01F687AF0119080711FD6E021207115F
S113B040FD0F11FDB6127E120711FD0F11FDB61290
S113B0507E120711FD0F11FDB612888AA6807E129A
S113B0600711FD0F11FD87B612864A26F10E08FD61
S113B07018088187F687AF01F687AF011908071111
S113B080FD6E03120711FD0F11FDB6127E1207119A
S113B090FD0F11FDB6127E120711FD0F11FDB61240
S113B0A0888A866E00120711FD0F11FD5E124A2672
S113B0B0F218088119080711FD6E05120711FD0F1A
S113B0C011FDB6126E00120711FD0F11FDB6121814
S113B0D008811908876E01120711FD0F11FDB612C0
S113B0E086B7120711FD0F11FDB61218088187CD1E
S113B0F0B00245B2C3CDA07E86CDA05D45B2C6CD1B
S113B100A07ECDB26F201445B2C3CDB27ECDA07265
S113B110A16F2679CDA072A16B2672A667CDA05D22
S113B120A66FCDA05D45019B35A8B6ACBAAD27048A
S113B130B6AC2710A001B7ACA680CDB257A680CD7F
S113B140B25720ECB6AD2731A180271C2504A68078
S113B150201645019BC601502702AF07A600F7AF92
S113B1600165021B26F8B6ADCDB257B6AD270AA1CC
S113B170802306A080B7AD20D955AE35ACA66FCDDF
S113B180A05DA66BCDA05D4F81A6022002A601CDD5
S113B190A05145B2A8CDB29CCDA0518145B2C0CD3D
S113B1A0B27ECDA072A16726E4CDA072A16F26DD88
S113B1B0B6ACBAAD2704B6AC271DA001B7AC4500A8
S113B1C0A8A600CDB073A600CDB23D55AAAF60AF1E
S113B1D060AF4035AA20DFB6AD270B4500A8CDB03F
S113B1E073B6ADCDB23D55AE35ACCDA072A16F26D0
S113B1F098CDA072A16B26914F8187CDB00245B244
S113B200C0CDA07E86CDA05D45B2C6CDA07ECDB218
S113B2106F209D87CE0150270EA0079EE7014501B0
S113B220A24FC70150200345019BCDA072F7AF0187
S113B2309EE6014A27059EE70120EF868187CD9B84
S113B240CF45019BF6CDA05DAF019EE6014A2705DF
S113B2509EE70120EF8681CDB213CDB024CDB0118D
S113B2604500A8CDB02E55AAAF20AF6035AA81CD38
S113B270A072B7ACB7AECDA072B7ADB7AF8187CD72
S113B280B002B6ACB7AEB6ADB7AFCDA07E86CDA09A
S113B2905DB6ACCDA05DB6ADCDA05D8187CDA07E01
S113B2A086CDA054CDA051817472616E73666572AF
S113B2B0206572726F722061626F7274696E6700CA
S10CB2C07A7A007A5A003F3F003B
S9030000FC
